:020000040000FA
:10000000B02B0020F90200000103000003030000F0
:1000100005030000070300000903000000000000C2
:100020000000000000000000000000000B030000C2
:100030000D030000000000000F030000110300008A
:100040005D05000013030000B90700001303000062
:100050001303000013030000130300001303000048
:100060001303000013030000130300001303000038
:100070001303000013030000130300001303000028
:1000800013030000B5050000130300001303000074
:10009000D905000013030000130300001303000040
:1000A00013030000130300001303000013030000F8
:1000B0001303000013030000000000000000000014
:1000C00013030000130300001303000013030000D8
:1000D00013030000130300001303000013030000C8
:1000E00013030000130300001303000000000000CE
:1000F00000000000130300000000000013030000D4
:1001000000000000000000000000000000000000EF
:1001100000000000000000000000000000000000DF
:1001200000000000000000000000000000000000CF
:1001300000000000000000000000000000000000BF
:1001400000000000000000000000000000000000AF
:10015000000000000000000000000000000000009F
:10016000000000000000000000000000000000008F
:10017000000000000000000000000000000000007F
:10018000000000000000000000000000000000006F
:10019000000000000000000000000000000000005F
:1001A000000000000000000000000000000000004F
:1001B000000000000000000000000000000000003F
:1001C000000000000000000000000000000000002F
:1001D000000000000000000000000000000000001F
:1001E000000000000000000000000000000000000F
:1001F00000000000000000000000000000000000FF
:10020000DFF80CD000F03CF900480047E92B000073
:10021000B02B002030B4044654E8000F0D4644E8EB
:100220000053002BF8D1156030BC704730B4044641
:1002300054E8000F40EA010544E80053002BF7D1D1
:10024000156030BC704730B4044654E8000F00EA33
:10025000010544E80053002BF7D1156030BC70470E
:1002600030B4044654E8000F80EA010544E8005326
:10027000002BF7D1156030BC704730B4044654E809
:10028000000F00EB010544E80053002BF7D1156087
:1002900030BC704730B4044654E8000FA0EB0105B1
:1002A00044E80053002BF7D1156030BC704770B4A0
:1002B00004464FF0000054E8006F0D68AE4207BFDF
:1002C00044E80023012044E800630E60002B1CBFBB
:1002D0000020F0E770BC704730B4044654E8000FCB
:1002E00088422CBF451A054644E80053002BF5D13F
:1002F000156030BC7047000006488047064800473C
:10030000FEE7FEE7FEE7FEE7FEE7FEE7FEE7FEE7C5
:10031000FEE7FEE7DD05000001020000004870472F
:10032000806100002DE9FE43994615468846074640
:1003300001AC022942D3002D40D000200290A8F148
:1003400001004FF0FF36009022E000FB057201FB38
:10035000057011464A469047002805DC54F82600EF
:10036000304444F8260013E060682A4600FB05711B
:1003700054F8040C00FB057007E00B7890F800C0FF
:1003800001F801CB00F8013B521E002AF5D176425C
:1003900054F8040C61688842D7DC4B462A4638463C
:1003A000FFF7C0FF54F8040C4B46A8EB0001401CBB
:1003B00000FB05702A46491EFFF7B4FFBDE8FE8327
:1003C00010B5431A934209D28318881803E010F835
:1003D000011D03F8011D521EF9D210BD40EA0103B0
:1003E0009B0703D009E008C9121F08C0042AFAD2EB
:1003F00003E011F8013B00F8013B521EF9D210BD99
:10040000D2B201E000F8012B491EFBD27047002256
:10041000F6E710B513460A4604461946FFF7F0FF03
:10042000204610BD421C10F8011B0029FBD1801A88
:10043000704710B5002200E0521C835C8C5CA34224
:1004400001D1002BF8D1D8B2E1B2401A10BD034659
:1004500011F8012B00F8012B002AF9D1184670473A
:1004600030B505460020034600E05B1C934205D2F0
:10047000EC5CC85C201A01D1002CF6D130BD000024
:10048000064C074D06E0E06840F0010394E80700E1
:1004900098471034AC42F6D3FFF7B6FEB0690000BF
:1004A000D069000070B58C1810F8015B15F00703D7
:1004B00001D110F8013B2A1106D110F8012B03E0FD
:1004C00010F8016B01F8016B5B1EF9D12B0705D405
:1004D0000023521E0DD401F8013BFAE710F8013B4E
:1004E000CB1A921C03E013F8015B01F8015B521E6A
:1004F000F9D5A142D8D3002070BD00F01F02012120
:1005000091404009800000F1E020C0F8801270475F
:1005100000F01F02012191404009800000F1E0201D
:10052000C0F80011704700F01F02012191404009FE
:10053000800000F1E020C0F8001270474907090E62
:10054000002806DA00F00F0000F1E02080F8141D0A
:10055000704700F1E02080F80014704770B54FF448
:100560008076304603F0B0FA114CB50560B13046E4
:1005700003F0B1FA0120C5F80803607920B9012021
:1005800060712168002088474FF48276304603F07E
:100590009BFA00280AD0304603F09DFA0220C5F8E5
:1005A00008032168BDE870400120084770BD0000C5
:1005B0005400002007480021C0F84011C0F8441141
:1005C000C0F84811C0F84C11C0F80011C0F804116F
:1005D00005F02AB90010014005F078B830B54FF0A9
:1005E000805000228300D0F83011C3F80C21C3F8EA
:1005F0001021624B1A60624B1B68624C2360604B97
:100600001B1D1B68241D23605D4B08331B68241DC4
:1006100023605B4B0C331B68241D2360584B103345
:100620001B68241D2360564B14331B68241D236054
:10063000534B18331B68534C20342360504B1C33EE
:100640001B68241D23604E4B20331B68241D236030
:100650004B4B24331B68241D2360494B28331B68F4
:10066000241D2360464B2C331B68241D2360444B00
:1006700030331B68434C40342360414B34331B6898
:10068000241D23603E4B38331B68241D23603C4BE4
:100690003C331B68241D2360394B40331B68241DE9
:1006A00023600124082902D1D0F8343113B108297C
:1006B00004D006E0354B3449196005E0D0F83431F8
:1006C00013B1082904D006E0314BFB21196005E085
:1006D000D0F8343113B1082908D00EE090F8583220
:1006E0002C48016863F30301016002E0D0F8343163
:1006F0001BB929494FF40070086028480168C907F0
:1007000002D06FF0010101602548016841F47001D9
:100710000160BFF34F8FBFF36F8F4FF01021D1F8FF
:100720000002002803DBD1F80402002822DA1D4B66
:100730001C601D480468002CFCD01224C1F8004243
:100740000568002DFCD0C1F8044201680029FCD0E6
:100750001A6001680029FCD0BFF34F8F10487C3825
:100760000168124A01F4E06111430160BFF34F8F49
:1007700000BFFDE70F490E48086030BD3805004056
:100780000404001020C50040488103008C5600403E
:1007900018F50040E40E004040960240000400407E
:1007A00088ED00E004E5014000E401400400FA05A2
:1007B0000090D003F80000200148006800470000C6
:1007C0005C00002002E008C8121F08C1002AFAD10C
:1007D00070477047002001E001C1121F002AFBD1C1
:1007E0007047000072B603F077FE00BF03F048FCCC
:1007F0000028FBD1134C606830B12088012101EB47
:10080000004011A103F066FD12480068C00700D047
:1008100000BE6068022806D32088022101EB004058
:100820000DA103F057FDBFF34F8F0A48E43801686C
:100830000D4A01F4E06111430160BFF34F8F00BF27
:10084000FDE7000094010020466174616C20657230
:10085000726F7200F0ED00E053797374656D207271
:1008600065736574000000000400FA050EB50021F0
:100870000091CDE901106A4644F20100FFF7B2FF92
:100880000EBD0000074B9B7823B12AB120B1006850
:10089000037C1BB1082070470720704741744261F8
:1008A00000207047C005002070B504F0EDFD104831
:1008B00000240B21047044700E4D817014206C6074
:1008C0002C706C70FFF719FE07211420FFF736FE1D
:1008D0001420FFF71DFE0848046007211120FFF7D0
:1008E0002DFE0548001F0068A860002070BD0000B4
:1008F000C005002064000020081501402DE9F843E0
:10090000DFF8709099F802305BB350B3052902D23A
:100910000720BDE8F88343691BB3437C012B22D039
:1009200000270446002588461646284600F036F87B
:10093000684605F09FF9C0B1012101700E4944607D
:100940000968C0E90218C0E904769DF8000089F83A
:100950000100002000F024F81420FFF7E4FD2846F1
:10096000D7E70820D5E70F46DBE70425002000F095
:1009700017F8F4E7C00500200415014006498978FE
:1009800039B130B1416921B100210174022104F073
:100990002BBF082070470000C005002000F002B8FF
:1009A00000F008B872B602480168491C016070473F
:1009B0007800002003490868401E086000D162B634
:1009C000704700007800002070B5054608680C46A6
:1009D000411C04D003F0A2FA206803F06FFA6068AB
:1009E000411C02D0002103F057FA2968A069C1F820
:1009F0002405607D227D29681043C1F86C05D4E987
:100A000000122868C0F81425C0F80C15207D0128B4
:100A100014D1A068411C02D0002103F03DFAE06827
:100A2000411C04D003F07AFAE06803F047FAD4E9F5
:100A300002122868C0F80825C0F8101570BD70B5FE
:100A4000054608680C46411C04D003F071FA206882
:100A500003F03EFA6068411C02D0002103F025FA41
:100A60002968A069C1F82405607D217D2A680843B2
:100A7000C2F86C05D4E900122868C0F80C15C0F85B
:100A80001425207D012814D1A068411C02D000212A
:100A900003F00BFAE068411C04D003F049FAE06867
:100AA00003F016FAD4E902122868C0F80825C0F845
:100AB000101570BD2DE9F0470546861C90460F467F
:100AC0004FF001090020FFF769FF1B4C20683860D8
:100AD000D4E90001401AA16804F21C47081A0EE08C
:100AE0000121384602F044FA01F094FF01463846ED
:100AF00002F03EFAD4E90001401AA168081A401C2D
:100B00008642EDD8B8F1000F03D0052065F38910B7
:100B100002E0062065F39F50A2682168114004EBB3
:100B20008101C8602068304420600020FFF738FF52
:100B30004846BDE8F08700008C07002030B482688A
:100B40000468531C8360A154D0E901128A4202D385
:100B500030BC03F064B830BC70470000034803C8E1
:100B6000814201D101207047002070478C0700208E
:100B700070B5816804468A7C002A4DD0C87C002864
:100B80004AD0121A0844D5B200F114016A1C13307D
:100B9000FFF716FCA068C17C491EC174A068817C67
:100BA000491E81748DB308221C49206903F02AF87C
:100BB000204602F0A9F98178C078814211D1A0685D
:100BC00017A2C17C431808212046143302F036FDD9
:100BD000204600F013F929462046BDE8704001F098
:100BE00015B8204600F01EF9204600F007F9A0686D
:100BF0000BA2C17C431808212046143302F01EFDCD
:100C00002046BDE8704000F003B92069BDE870409F
:100C1000044A03A102F0F6BF70BD0000F80D000009
:100C200025730000E45F000070B504468068827C94
:100C3000C17C521A12F0FF053AD0084400F11501A8
:100C40002A461430FFF7BCFBA068817C491E8174E2
:100C5000204602F059F98178C078814214D1A06809
:100C600014A2C17C431808212046143302F0E6FC8C
:100C7000114A10A1206902F0C5FF6D1EE9B220469D
:100C8000BDE8704000F0C2BF204600F0CBF820461F
:100C900000F0B4F8A06807A2C17C431808212046E0
:100CA000143302F0CBFC2046BDE8704000F0B0B831
:100CB00070BD000025730000E85F00002DE9F041E1
:100CC000044680680F46D0F83C11C27C11F0010642
:100CD000817CA1EB0203DDB20AD07F2901D3002D74
:100CE0007ED0A068C17C08440021077566B113E07E
:100CF0007F297CD2002DF4D0831803F114012A46F9
:100D0000481CFFF75DFBECE7A068827C521CD2B266
:100D10008274A068143281544DB3204602F0F4F876
:100D20008178C07881420ED1A06832A2C17C43187C
:100D300008212046143302F081FCA81BC1B22046D2
:100D400000F064FF21E0204600F06CF8A06829A2C2
:100D5000C17C431808212046143302F06FFC204662
:100D600000F056F80121204601F02EF80DE03EB1CA
:100D7000A068827C521CD2B28274A0681432815462
:100D80003A461DA1206902F03DFFA168C87C401CC5
:100D9000C874204600F027FF0028204603D0BDE895
:100DA000F04100F03FBF01F06AFA00281FD0204652
:100DB00002F0AAF80546C078A978401A401EC1B2D0
:100DC000204600F0B1FE204600F02CFFE878A9781C
:100DD000401AC1B2204601F003F82878401E00E016
:100DE00005E0C1B22046BDE8F04100F0EDBFBDE82E
:100DF000F081000025730000256300000069024AAD
:100E000002A102F0FFBE0000DC5F000025730000BD
:100E10000069024A024902F0F5BE0000D35F0000FB
:100E20000C0E00000069024A024902F0EBBE00000D
:100E3000D05F00000C0E00002DE9F04F4FF00009CC
:100E40009DB005464E464C46CDF8149000F07EFD10
:100E5000284601F039FB284600F072FE284600F0D3
:100E6000C2FE10B9284600F0DDFEAA680C2308A9CE
:100E700001A8143201F024FF0346019840B15BB190
:100E800050A20221284602F0D9FB1DB0BDE8F08F28
:100E9000284600F0C7FEF8E7514850490027A1EB6B
:100EA00000080DF1200A834613E008D34DA00090FE
:100EB00051A202212846089B02F0C0FBE5E70BEB9C
:100EC000C704606801685AF82900FFF7B2FA18B140
:100ED0007F1CB7EBD80FE8D94FF0000BCDF868B006
:100EE0006068C7680FB1A9684860606809F10104CB
:100EF0004FF0000880680DF158090690019884426F
:100F000037D25AF824003EA1FFF793FA50B35AF8AB
:100F100024003CA1FFF78DFA20B3424608F10108F6
:100F20001AAB2146CDF80090069800F0CBFCB8F142
:100F3000000F1ED01A98E0B101685AF82400FFF79C
:100F400078FA0028DAD11A98C16829B1A8F101010C
:100F5000DDF818B02646059180684FF00008641C43
:100F60000690CBE7A868D0F83C1141F00201C0F828
:100F70003C11BBF1000F12D0CDF800901AAB3146F6
:100F80005846059A00F09EFCA9681A980AEB86025A
:100F900048600199C368891B284698470AE027B131
:100FA00008AA28460199B84704E018A20221284659
:100FB00002F044FBA868D0F83C1121F00201C0F80F
:100FC0003C1162E76E6F74207465726D696E6174B6
:100FD00065643A2025630D0A00000000106A0000D5
:100FE000D06900003A20636F6D6D616E64206E6F92
:100FF0007420666F756E6400257325730D0A0000FA
:101000002D6800002D2D68656C700000506C6561C6
:1010100073652073706563696679206120737562FA
:10102000636F6D6D616E642E0D0A00008068D0F8EC
:101030003C01C0F3C00070472DE9F0410446C06890
:101040008EB00D460026C068324601A903F04FFB62
:1010500018B100200EB0BDE8F0816DB1019803F029
:10106000F9FAA168D1F82C01401CC1F82C0100F05C
:101070000700012879D10126204601F045FF0546E9
:101080008078012804D9401EC1B2204600F0A8FE95
:101090002878012804D9401EC1B2204600F0B6FDD0
:1010A0002046FFF7ABFE2EB131A20221204602F00E
:1010B000C5FA5AE04FF000080023082202A901985F
:1010C00003F0D7FA04980590BDF80C00ADF81800AD
:1010D000BDF80E00ADF81A008DF81D8002980827A3
:1010E00000F00300012802D0022818D032E0029854
:1010F0003B46860AC0F3C2008DF81C00029808A97E
:10110000C0F38315AA00019803F0B3FA2069009098
:1011100005AB2A4608A9304603F0F2F91AE0029816
:10112000850DC0F3C2008DF81C00082D01D22E469B
:1011300000E008263B46324608A9019803F099FAD8
:101140003744AD1B05AA314608A8236903F0C6F849
:10115000002DEAD1019803F07DFAE068002201A990
:10116000C06803F0C4FA0028A6D0012072E700008E
:101170004C6F7374206C6F6773202D20696E6372DF
:1011800065617365206C6F67206261636B656E6477
:101190002071756575652073697A652E0D0A0000EA
:1011A00030B4406804682469A44630BC60477CB50C
:1011B00000260446019601AB012269462046FFF74E
:1011C000EFFF019800281CD09DF800007F28F2D87E
:1011D00003F08CFAA068417821B1012961D002297D
:1011E00063D167E0217E9DF80050A9420DD1807C3B
:1011F0000028204606D0FFF71FFE0221204600F0FF
:10120000C7F87CBD00F00EFDF7E7092D1CD004DC0B
:10121000002DD0D0082D04D11FE01B2D12D07F2D22
:1012200024D0FFF77BF80068405D10F03E0FC2D07D
:101230002046FFF7FBFE9DF8001000B32046FFF7A5
:101240003DFDB8E7012133E02046FFF7EFFE00281F
:10125000B1D0204600F0B6F8ADE72046FFF7E6FE35
:101260000028A8D02046FFF783FCA4E72046FFF71C
:10127000DDFE00289FD02046FFF7D6FC9BE7A26842
:10128000907C7F2897D2D07C1318401CD07419759D
:10129000A068C17C08440675A068817C491C8174E3
:1012A00089E79DF800105B2901D0002100E00221B0
:1012B000417080E7002141702046FFF7B7FE00280B
:1012C0009FD09DF8000041380C28BAD2DFE800F02A
:1012D00007090E2D064C0650060606546BE7012141
:1012E00000E00021204600F0DDFF64E7204601F029
:1012F0000BFE054600786978884203D1A978EA7820
:1013000091429ED0697988424FF00101204606D172
:1013100000F00AFC6979204600F078FC01E000F05A
:1013200053FDA068C17C491C15E0204601F0ECFD8E
:1013300005460078A979491C884202D1A97801297B
:101340008AD001284FF00101204606D000F05EFC53
:10135000A068C17C491EC1742DE700F041FD697988
:10136000204600F031FDF3E7204600F0E9FB22E7DC
:10137000204600F00EFC1EE7A068D0F83C210121B9
:101380009143D0F83C2161F30002C0F83C2112E700
:101390008268022911700BD1826800211175826860
:1013A000D1748268917403A20321036802F046B9E4
:1013B0007047000025730000002801D0FFF732B805
:1013C000704700002DE9F04FA7B04FF00008054628
:1013D000CDF82480CDF8188080684746817CC1F123
:1013E0007F01C9B25FEA010B7BD0C27C00F114011E
:1013F0009430FEF7E5FFA8680024C17C084480F81B
:101400009440FEF78BFF21900168A8680C23C27CF2
:101410000244D27C895CC0F83841AA6801F0010915
:1014200012A920A8943201F04BFC1298FFF7C4FFD8
:10143000C6B2A2461F940C94209818B14844401E8E
:10144000B8426AD8B9F1000F01D0002605E012A811
:1014500050F82700FFF7B0FFC6B200240DA82246BF
:101460000090641C1FAB3946504600F02BFA1F98C1
:1014700000286BD0016812A8324650F82700FEF70A
:10148000EFFF00280C9802D00028E7D05EE0D8B12A
:101490001F980068FFF790FF0699C0B2884200D9F4
:1014A0000690BBF1000F2BD022A800900CAB424657
:1014B0003946504600F006FA1F98006882190C98C9
:1014C00000688319002015E0601E09901F980068CD
:1014D000FFF772FFC0B20690801B584510DAC0B209
:1014E0000DE07FE013F800C0614506D1401C10F00C
:1014F000FF0010D0115C0029F4D1834500D9834648
:101500001F98B4F101080C90A8D263A204212846C8
:1015100002F094F81AE0FF20EFE700240DA822461D
:101520000090641C1FAB3946504600F0CBF9ECB379
:101530001F98002856D0016812A850F82700FEF71F
:1015400078FF0028EAD11F98D0F808A0BAF1000F60
:1015500009D01F9838B120997F1CFFB201EB090018
:101560008742FFF469AF0C9800283BD009984146A8
:1015700040455FD19AF8000038B10DA80A460090A6
:101580000CAB3946504600F09DF90C980068FFF707
:1015900013FFB04206D00C985A46006881192846BD
:1015A00000F078FA2198A968026800E01DE0C87C84
:1015B0000B181B7DD25CD2071DD0897C884211D2CA
:1015C000284601F0A1FCA9688478C87C401CC87436
:1015D000284601F099FC8078A04227D101212846B5
:1015E00000F0F2FB27B0BDE8F08F2BA204212846C3
:1015F00002F024F8F6E7D1F83C01C00711D0D1F889
:101600003C0120F00100C1F83C0120212846FFF7F1
:1016100055FBA868D0F83C1141F00101C0F83C111D
:10162000E0E720212846FFF749FBDBE7284600F0EA
:10163000F9FAD7E700212846069A03F05BFE0DF180
:101640003409099C0EE01FAB224639465046CDF8BE
:10165000009000F037F91F98069A0168284603F0B9
:1016600049FE641C4445EED917A2032128462B6885
:1016700001F0E4FFAB6816A208212846143301F0FC
:10168000DDFF284600F06AFB0C985A460068811975
:10169000284600F0FFF9A5E75461622066756E6385
:1016A00074696F6E3A20636F6D6D616E6473206351
:1016B0006F756E746572206F766572666C6F776594
:1016C000642E0D0A000000000D0A257300000000C2
:1016D00025730000002806D08868D0F83C1141F03E
:1016E0002001C0F83C11704770B5044640680D46B3
:1016F00090F8280030B1A0680068FFF73FF908B102
:1017000008280CD1012685B1606902F06FFA616882
:1017100000220831606902F025FA08B1062070BD88
:10172000606880F82960002070BD606890F828002B
:1017300048B9074A0021A068FFF7A4F861680028AB
:1017400081F82860F0D12046BDE8704003F0FABE71
:10175000B156000070B5044640680D4602606068EE
:1017600000224360606880F82820606880F82920A3
:10177000606820220830FEF723FE2C61074A2946C4
:10178000606902F0EFF9050005D1E06803F0E7F9C0
:10179000206903F0E4F9284670BD0000D758000026
:1017A0001A60C0681A4603F018B910B504464069BB
:1017B00002F01CFAA0680068BDE81040FFF7DEB830
:1017C0007CB51A60044600691A4603F044F9050026
:1017D00025D16069134A0178515C19B1001D03F0ED
:1017E00023FD02E00C3003F0A9FBC0B9FF200090FC
:1017F00001236A4601A9206903F079F978B90098B4
:101800000199C2B2606902F0E1F90546606890F89A
:10181000290020B11DB92069009903F055F9284627
:101820007CBD0000400000202DE9F8431E4615460F
:101830008846074600241BE0786808EB04016B46E5
:101840000268D2F80CC02A46E047009804442D1ADA
:1018500070B9B868017803290AD000BFD0F83C11EC
:101860008906FBD5D0F83C1121F02001C0F83C11CD
:10187000002DE1D1002E01D000983060BDE8F88342
:1018800070B5084C050009D010342168002907D034
:1018900008682060496828468847F6E70834F4E776
:1018A00070BD00005C050020054A012120B101281F
:1018B00005D19170FFF7E4BF51700020FAE770473F
:1018C0005C0500202DE9F05F1C460A9E15464FF08E
:1018D000000959B180B3017839B3426831462846CE
:1018E00090473068D8B12660BDE8F09F144915488C
:1018F000A1EB0008B5EBD80F11D2DFF84CA0002601
:10190000834609E00BEBC607786801685AF82500A2
:10191000FEF78FFD30B1761CB6EBD80FF2D3C4F8CA
:101920000090E1E778682060DEE7406800EB021095
:10193000016809B11860D7E7FFE7C3F80090D3E763
:10194000106A0000D0690000FC0000202DE9F04181
:10195000856806460024287D002812D0A046FEF7A0
:10196000DDFC0746D0F8000004F1140104F1010485
:10197000695CE4B2415CC90705D0002CF4D185F85C
:101980001480BDE8F081641E14F0FF040FD0A87C21
:10199000021B04F11400291805F11400521CFEF773
:1019A0000FFDB168887C001B8874B168C874B26888
:1019B0003D68937CD01813300446002102E0491C96
:1019C000C9B2401E0778EF5DFF07F8D18442D8D036
:1019D0005B1A143302F80380B268907C401A90744A
:1019E000B168C874CDE700002DE9F05F2648416872
:1019F000F1B3DFF898B00E688146DBF800408768E5
:101A00008078E11B21F07F45ED1CB0B9DFF88080C4
:101A10004FF48030C8F84403C8F804031120FEF7DF
:101A20006CFD1120FEF774FD4FF0010AC8F800A00C
:101A30002F2003F00DF989F802A0B54200D23546F7
:101A4000124BE8193C3320F07F401860DBF800109F
:101A50005A46091B21F07F41001B20F07F40C91C22
:101A600081420FD9106818602F2003F0F1F800E0D0
:101A700004E0BDE8F05F1120FEF755BDBDE8F05F62
:101A800003F002BDBDE8F09F640000200415014092
:101A9000001001402DE9F0410446806815460F46CC
:101AA000827CC17C531A2A44DEB27F2A37D8002DAB
:101AB00035D0084400F1140105F114021044721CE1
:101AC000FEF77EFCA0682A46C17C084439461430E3
:101AD000FEF776FCA0681430FFF76EFCA16811A237
:101AE0008874A068C17C431808212046143301F093
:101AF000A5FDA068C17C2944C174204600F073F89C
:101B000018B9204600F0BBFB10B1204600F08AF85F
:101B1000002E04D02046BDE8F04100F01FB9BDE81A
:101B2000F081000025730000002904D00A460069F6
:101B300001A102F067B870471B5B256442000000FA
:101B400070B5054601F0E0F90446007861788842F6
:101B500003D1A078E17888421AD0E178A078814258
:101B600004D9081AC1B22846FFF7DEFF2078617851
:101B7000884205D9401AC1B2284600F047F804E06F
:101B8000081AC1B2284600F01FF9A868817CC17408
:101B900070BD70B5054601F0B7F90446017880794B
:101BA000401C814202D1A07801281BD0A0780128D6
:101BB00004D9401EC1B2284600F012F92078A1795C
:101BC000884206D9401A401EC1B2284600F01EF8CD
:101BD00005E0081A401CC1B2284600F0F5F8A968D3
:101BE0000020C87470BD10B504460068FFF7E4FB20
:101BF0000146A068C27C407B1144B1FBF0F200FBBF
:101C0000121008B1002010BD012010BD002904D021
:101C10000A46006901A101F0F5BF70471B5B25640E
:101C2000440000000069024A024901F0EBBF0000D5
:101C3000D65F00000C0E00002DE9FC47002604468C
:101C40008DF8046080683546B146B04680219430F6
:101C5000FEF7DDFB4049206901F0D4FF206901F067
:101C6000DEFF00276B46012201A92046FFF798FA04
:101C70000098D8B19DF804001B2806D0A16891F8FF
:101C800094101B29EED152281FD0A26808F19401AC
:101C9000505408F1010000F0FF08B8F1090F0AD90B
:101CA000A168042081F89490BDE8FC872A494FF68A
:101CB000C0100D31884700980028D3D17F1CBFB2D7
:101CC000B7F57A7FCED30D20EEE7A16808F1940036
:101CD0004A4601F80090A16891F895005B2803D06E
:101CE00081F894200B20DFE702206FF02F0309E03A
:101CF00005EB850503EB4505401C3D44C0B2ADB284
:101D0000802808D200F19407CF5D3B2FF0D1401C12
:101D1000C0B2802809D30C20C6E700BF06EB8606B8
:101D200003EB46063E44B6B2F1E700F19407CF5DFF
:101D3000002FF3D1FA20FA2E01D9087200E00E72BA
:101D4000FA2D02D9A168887201E0A0688572A068A6
:101D500080F894200020A7E7F45F000070B50546E6
:101D600001F0D2F804468078E178884201D101265A
:101D700000E000262846FFF736FF18B9284600F095
:101D80007EFA10B12846FFF74DFF1EB1607821782A
:101D9000401A12E0E078A178401AC1B2284600F05B
:101DA0001FF820786178884206D9401AC1B22846C7
:101DB000BDE8704000F008B8081AC1B22846BDE876
:101DC0007040FFF723BF0000002904D00A460069D5
:101DD00001A101F017BF70471B5B256443000000A1
:101DE000002904D00A46006901A101F00BBF704729
:101DF0001B5B25644100000010B50021024801F082
:101E0000CDF880F3100010BDA80B00200E4910B5CE
:101E10000A784C780023A24212D0521CD2B20A7027
:101E2000022A00D10B70084A0B780C3252F823209A
:101E300002608868104420F07F408860012010BD57
:101E40000360002010BD00006400002030B44FF09B
:101E5000805250690C49401E886012690B4C5043F7
:101E6000C1E900020A4D0246C8601368A34208D0C7
:101E7000AB4203D102F58072CA60F6E730BC02F0D3
:101E800005BC30BC704700004C050020A55A5AA57F
:101E900000005AA51CB5012905D08168D1F83C1174
:101EA000C1F3400131B102B00022BDE8104011463B
:101EB00001F0ECBB536804A1CDE90013136808A23C
:101EC000022101F0BBFB1CBD20756E6B6E6F776E3F
:101ED00020706172616D657465723A2000000000C7
:101EE00025733A257325730D0A00000010B5034CC5
:101EF000206802F0CBFB2068E06010BD4C0500209C
:101F00002DE9F043194D0746194E2C68E86891B049
:101F1000A04224D12068B04221D016A205E020685A
:101F2000B04209D0484507D01AA20421384601F032
:101F300085FB11B0BDE8F0830020414604EB800230
:101F400012790A54401CC0B23E28F7D96B4617A23A
:101F50000821384601F072FB04F5807402E0DFF8D6
:101F60005490E846E868A042D9D2E2E74C05002048
:101F7000A55A5AA5506C65617365207772697465BE
:101F800020736F6D657468696E672066697273741B
:101F90002E0D0A00436F727275707465642064615F
:101FA000746120666F756E642E0D0A0025730D0A2C
:101FB0000000000000005AA52DE9F8431646074628
:101FC000022906D233A00090136838A24FF0020114
:101FD00006E00AD937A00090136834A24FF004013C
:101FE000384601F02BFBBDE8F8837068FEF71AFA5B
:101FF00005463E2808D901B03846BDE8F0433E23E7
:1020000037A2022101F01ABB444CDFF81481E068CA
:1020100001684A1C1CD0414503D042A24FF0020186
:102020000AE015D1226800F50071A1EB0201B1F5BB
:10203000805F06D946A204213846BDE8F84301F086
:10204000FDBA4F4902F03AFBE06800F58070E060AD
:1020500074684C4E0346021D012030604A486D1CD6
:1020600001680029FCD0002106E0675C42F821707D
:102070000768002FFCD0491CA942F6D3002131602B
:1020800001680029FCD041461846BDE8F84302F03B
:1020900015BB00002062616420706172616D65741F
:1020A000657220636F756E740D0A000025733A2502
:1020B000730000002062616420706172616D65745C
:1020C000657220636F756E74202D20706C6561736E
:1020D00065207573652071756F7465730D0A000056
:1020E000546F6F206C6F6E6720737472696E672E09
:1020F00020506C65617365206C696D697420656E34
:10210000746572656420737472696E6720746F20E1
:1021100025642063686172732E0D0A004C0500204F
:10212000A55A5AA5466C61736820636F7272757008
:102130007465642C20706C656173652065727261D2
:1021400073652069742066697273742E0000000044
:102150004E6F7420656E6F7567682073706163657C
:10216000202D20706C656173652065726173652038
:10217000666C6173682066697273742E0D0A0000C4
:1021800000005AA504E5014000E401402DE9F05F9C
:1021900017460E00814670D013B1F9B2FFF714FE56
:1021A0000024FEF7BBF88246006800E0641C315D45
:1021B000415CC907FAD100253046FFF7FDF8D9F890
:1021C0000810001B4A7BD11B814228D306EB040870
:1021D00005E000BF18F805100A290CD06D1C8542D7
:1021E000F8D33119D9F8100001F00CFD4846BDE8CC
:1021F000F05FFFF717BDD9F8100001F010FD414660
:1022000000232A464846FFF70FFB2C444846641C2F
:10221000FFF708FDF9B24846FFF7D6FDE1E78B4628
:10222000DAF8001006EB040818F805000B5CDB0771
:1022300002D0AB460A2804D0E819904201D26D1CA6
:10224000F2E7D9F8100001F0EAFC414600235A46B3
:102250004846FFF7E9FA5C44DAF8000000E0641C45
:10226000315D415CC907FAD14846FFF7DBFCF9B2A2
:102270004846FFF7A9FD9EE7FFE7BDE8F09F10B5D0
:1022800004460068FFF798F80146A068827C407B0E
:102290001144B1FBF0F200FB121008B1002010BD98
:1022A000012010BDFEB50026044600960196029658
:1022B0008068E9B3D0E94D128A4271D0D0F830017C
:1022C00000286DD02046FFF764FCA068D0F8385194
:1022D000002D68D0002309226946284602F0C9F97A
:1022E000A1689DF808500098C1F83801A068002343
:1022F0000922D0F83801694602F0BBF9A1689DF8BF
:1023000008200923D1F838011431521C02F0B1F928
:10231000A1689DF80800C874A1689DF80800887439
:102320009DF80800A84202D22046FEF767FD00E0B3
:102330000BE0A3682BA208212046143301F07EF99C
:102340002046FFF750FC60BB42E0D0F8380100287F
:1023500046D02046FFF71DFCA06800230922D0F8D4
:102360003801694602F085F9A0680199C0F8381172
:10237000A0680029857CB9D19430FFF71DF80028AA
:10238000A06805D000F194011430FEF760F800E079
:102390000675A0681430FFF70FF88DF80800B7E74E
:1023A0001EE01AE0FFE71430FFF706F810F0FF0513
:1023B000A068D0F83011C0F83811A06805D000F13D
:1023C00014019430FEF743F890E780F894608DE7AD
:1023D0002046FFF754FF002802D02046FFF722FCDA
:1023E000FEBD000025730000FEB50D468168044661
:1023F0000026D1F8300138B300230922694602F0E3
:1024000038F90195A06800230922D0F83001694607
:1024100002F035F90196A068D0F830110091807C67
:102420008DF80800A068C0F83051002309226946E1
:10243000284602F024F9A168092328468A7C143131
:10244000521C02F01CF9FEBDC1F83051A068C0F862
:10245000345100960196A068807C8DF80800E4E76E
:10246000FEB504468068D0F83461002E28D00023E1
:1024700009226946304602F0FCF8A168019800255F
:10248000C1F83401009501952B4609226946304672
:10249000029502F0F4F8304602F0BDF8A168D1F8D8
:1024A000340170B100230922694602F0E2F8009578
:1024B000A06800230922D0F83401694602F0DFF851
:1024C000FEBDC1F83051FEBDFEB504468068143033
:1024D000FEF772FF10F0FF05A0684FF00006C0F88D
:1024E000386133D0A068D0F83001E0B10023092270
:1024F000694602F0BEF89DF80820AA4213D1A068F0
:10250000092300F19401D0F83001521C02F0B1F817
:10251000A06800F194011430FDF78BFF0028A0683B
:1025200080F8946012D000260A352946606902F0CE
:1025300042F80100204604D003B0BDE8F040FFF7A8
:1025400053BFFFF78DFF761C082EEED3FEBD0000B3
:102550002DE9FC5F0E008346DDE90C47C6F1000063
:1025600098469246814600D40846012503E000BF04
:1025700090FBFAF06D1C5045FADAA84500D94546A3
:1025800024B1002E01DB780700D5641EB80702D500
:10259000B8F1000F0AD0F80708D13CB1A54205D226
:1025A00020215846641EFEF7C9FAF6E7002E02DA2B
:1025B0004E462D2102E0780703D52B215846FEF721
:1025C000BDFA07F0030002280BD1B8F1000F08D1C3
:1025D0003CB1A54205D230215846641EFEF7AEFA42
:1025E000F6E7CDE90047434652463146584603F0E8
:1025F000E7FABDE8FC9F000070B50D460446006890
:102600004FF4887102F0E7FA4FF49071206802F0FD
:10261000E2FA4FF49271206802F0DDFA4FF4A271F1
:10262000206802F0D8FA20681249C0F80413206824
:102630006907000B40B2090E002806DA00F00F000F
:1026400000F1E02080F8141D03E000F1E02080F8A4
:10265000001420680121000B40B200F01F029140DD
:102660004009800000F1E020C0F88012C0F800119D
:1026700070BD00001003020002460020126893079C
:1026800002D0530702D47047500714D502F003005C
:10269000012802D002280CD105E0C2F383100B6898
:1026A000801C184404E00223086803EB9252104493
:1026B000086001207047086800EB9253C2F389104C
:1026C000401CEEE70268134602E08A4204D012681A
:1026D000002AFAD10B600160704700002DE9F04735
:1026E000394E002780463D46DFF8E090D6F804A03A
:1026F00057E003D00446D0F81C8035E099F800205C
:1027000002EB4201521CD2B289F8002009EBC10150
:1027100099F80230091D9A4201D189F800504868A1
:102720000A780446012A12D0022A02D0032A3BD199
:1027300008E003F029F800B10127257434E005749E
:10274000C06900E070680028F9D170602CE0207C3E
:1027500050BB88686060C868A0600869E06048692C
:10276000A061F07800B165606268B168184B501ADA
:1027700020F07F40984202D2A168084406E0881AFF
:10278000A16820F07F40814202D9081A206000E051
:10279000256065600120A56020742046E56102F097
:1027A000D5FFB8F10000A4D199F8001099F8010004
:1027B0008142A3D117B97168514502D00120BDE80B
:1027C000F0870020FBE7000064000020C005002027
:1027D000FFFF7F001CB5012905D08168D1F83C11AD
:1027E000C1F3400131B102B00022BDE810401146F2
:1027F00000F04CBF536804A1CDE90013136808A290
:10280000022100F01BFF1CBD20756E6B6E6F776E92
:1028100020706172616D657465723A20000000007D
:1028200025733A257325730D0A0000002DE9F74F33
:1028300082B0154602980F004FF00006C068007A7B
:10284000009058D0072248A12868FDF709FE78B10A
:10285000082247A12868FDF703FE002830D02B6826
:1028600045A2029805B00221BDE8F04F00F0E6BE97
:10287000012F02D0022F08D008E0029805B044A230
:10288000BDE8F04F022100F0D9BE0126DFF8188123
:10289000002400BF58F824100A226868FDF7E0FD04
:1028A00010B1641C052CF5D3052C06D004F0FF09EB
:1028B0000224002E54D0002419E03CA26B68D0E71B
:1028C000012F4FF00009F6D0012449E04A46214685
:1028D000009800F0DDFA48B90021204601F0EEFD35
:1028E00003463AA20221029800F0A8FE641C01F0FF
:1028F00093FDA042EAD805B0BDE8F08F4FF0000A82
:1029000055F824B001F088FD8046002609E000213A
:10291000304601F0D3FD20225946FDF7A1FD90B1CC
:10292000761C4645F3D3464506D155F8243030A2EF
:102930000221029800F082FE4A465146009800F0BB
:10294000A7FA10B10BE0B246EDE70021504601F0C6
:10295000B5FD03461DA20221029800F06FFE641C23
:10296000BC42CBD3C7E70000656E61626C650000B6
:1029700064697361626C6500556E6B6E6F776E2073
:102980006F7074696F6E3A2025730D0A00000000A5
:1029900042616420706172616D6574657220636F5D
:1029A000756E742E0D0A000080000020556E6B6E4F
:1029B0006F776E207365766572697479206C6576C1
:1029C000656C3A2025730D0A000000004C657665A1
:1029D0006C20756E617661696C61626C6520666FF2
:1029E00072206D6F64756C653A2025730D0A0000C6
:1029F000556E6B6E6F776E206D6F64756C653A25E2
:102A0000730D0A00C068012141727047C06800213F
:102A1000417270472DE9FF410026234800F0A2FAD9
:102A20002148001F074600F09DFA204C6068009086
:102A3000A56800E000986946284004EB80000C304F
:102A4000FFF71AFE0028F5D101AA009901EA050353
:102A500004EB8303491CDB6842F82030401C0091E2
:102A60000228F2D3019800F0030001280BD00228BD
:102A700010D10198032101EB90500099BDF80A6034
:102A800001EB900005E00198BDF80A60C0F38310E7
:102A900008440090384600F062FA08B1009860607F
:102AA00004B03046BDE8F081A40B00208C07002064
:102AB0002DE9FE4F814601F0AFFC0746D9F80C0026
:102AC00090F80880407A20B91FA20221484600F001
:102AD000B5FD22A324A20821484600F0AFFD2AA29A
:102AE0000821484600F0AAFD002429E001231A46E7
:102AF0002146404601F09AFC8246002301222146ED
:102B0000404601F093FC0546032801D2064600E04A
:102B100003260121204601F0D1FC0346AE4201D23A
:102B200029A200E027A2294850F8261050F82A00D0
:102B30008DE8070026A20821484600F07FFD641CAE
:102B4000BC42D3D3BDE8FE8F4C6F677320617265C2
:102B50002068616C746564210D0A00006D6F6475F6
:102B60006C655F6E616D6500252D343073207C20AF
:102B700063757272656E74207C206275696C742D49
:102B8000696E200D0A0000002D2D2D2D2D2D2D2DCF
:102B90002D2D2D2D2D2D2D2D2D2D2D2D2D2D2D2D65
:102BA0002D2D2D2D2D2D2D2D2D2D2D2D2D2D2D2D55
:102BB0002D2D2D2D2D2D2D2D2D2D2D2D2D2D2D2D45
:102BC0002D2D0D0A000000002A00000080000020CA
:102BD000252D343073207C20252D3773207C202533
:102BE0007325730D0A0000008AB04FF400410020E5
:102BF00001F0CAFB08B1FDF739FEFDF755FE08B13B
:102C0000FDF734FE00F070FF002420B1852802D0CB
:102C1000FDF72CFE02E0002000F080FFFFF716F920
:102C200020221C4901A8FDF7CBFB062001900820BB
:102C3000029003200090174801238DF818401A468F
:102C400001A91C3800F066FE08B1FDF70FFE11481F
:102C50001C3800F015FF08B1FDF708FE0E4C606847
:102C600003280FD32088052505EB00400BA101F0B8
:102C700031FB6068032805D32088104905EB00402C
:102C800001F028FB01F0FCF902481C3800F0BEFE00
:102C9000F8E70000945D000094010020466C617329
:102CA000687772697465206578616D706C652073F2
:102CB0007461727465642E0D0A0000008461000066
:102CC0002DE9FF4F4FF0000881B014468B46814636
:102CD000C246C0F800802578002D71D0FDF71EFB9C
:102CE00000900068405DC00702D004F801AB84E0AA
:102CF000D9F800008300401CC9F800004BF80340DD
:102D000015E02678002E78D0B8F1000F05D1222EDC
:102D100010D0272E0ED05C2E1ED0B04514D12046E8
:102D2000FEF74AFB0246611C2046FDF749FB4FF0C7
:102D30000008E6E72046FEF73FFB0246611C2046FE
:102D4000FDF73EFBB046DCE7B8F1000F50D05C2E3B
:102D500061D16078404508D12046FEF72DFB024640
:102D6000611C2046FDF72CFB55E030281CD10027C4
:102D70000225605DA0F13001072906D86D1C41EAEB
:102D8000C701EDB2CFB2052DF3D3022D0CD92046E9
:102D9000FEF712FB421B61192046491E921CFDF7EB
:102DA0000FFB04F8017BACE778281ED10027022531
:102DB000605DA0F13001092903D841EA07100DE058
:102DC00021E0A0F16101052901D8573804E0A0F104
:102DD0004101052907D8373840EA07106D1CEDB2CC
:102DE000C7B2042DE4D3022DD1D8B8F1000F12D10F
:102DF00000980068805DC0070DD0D9F800100498D5
:102E00008142FFF468AFD9F8002040464BF822A079
:102E100005B0BDE8F08F641C73E72DE9F047C78863
:102E20000446181D16468946B0FBF7F1B0FBF7F2D1
:102E300007FB12009A193A44D21CB2FBF7F2DDF8F4
:102E400020A001E02468491E0029FBD13D1A8846D4
:102E5000B54216D818E0BAF1000F05D0211809EBD9
:102E600008002A46091D04E0204409EB08012A460F
:102E7000001DFDF7A5FA00202468761BA844B74280
:102E800001D9354600E03D46002EE4D1BDE8F0878B
:102E900070B5144600230D4606461A4601F0C6FAE0
:102EA000844201D9002070BD22462946304601F0F7
:102EB000E3FA012070BD000030B5024669B101F0AF
:102EC000ABFA0021084C0BE001EB410304EB830358
:102ED00015685B88AB4202D11160002030BD491CEF
:102EE0008142F1D3052030BD1C01002010B50C46F5
:102EF0000021E16061600349A160012101F0DEFA77
:102F0000206010BD7460000070B58468006804F132
:102F10000805FEF751FAC1B2A971E07C6A7908444C
:102F2000B0FBF2F302FB13035B1C2B70E07C084444
:102F3000B0FBF2F35B1CAB70A07C0844B0FBF2F377
:102F40005B1CEB70A07C0844B0FBF2F102FB1101AA
:102F5000491C6970284670BD002100F00FB800219F
:102F600000F012B8012100F01EB8012100F011B8E4
:102F700008B56A46FDF781F9009808BD08B56A46AC
:102F8000FDF761F9009808BD08B56A46FDF75BF9E1
:102F900008BD08B56A46FDF749F908BD08B56A4697
:102FA000FDF738F908BD08B56A46FDF73FF9009806
:102FB00008BD08B56A46FDF76DF9009808BD70B503
:102FC000044600252846FDF7E9FC21686268086888
:102FD00090420ED9401E08600178238BE26801FB05
:102FE0000325227A2168101AC0B20A79824200D2DF
:102FF00008710020FDF7D4FC284670BD70B5054669
:103000000C460020FDF7CAFCE868298B201AB0FBAB
:10301000F1F12A681068431C13600170BDE870402C
:103020000020FDF7BDBC10B530B1017A42680368DD
:10303000891AC9B21A6006E00E2010BD03681A682A
:10304000541C1C601170491EC9B2F7D200680021DF
:103050000171084610BD00002DE9F0470646806862
:1030600088B0D0F83C01C0F3400038B108B0304619
:10307000BDE8F0470022114600F008BB012907D93E
:1030800008B03046BDE8F0471DA2022100F0D6BAD4
:103090002049DFF884A0A1EB0A001C21B0FBF1F568
:1030A000002428E0C4EBC4010AEB81034FF00009BF
:1030B0001F68D3E901103A793F78411AB3F81880B4
:1030C000C01B5B69C0B2642712FB07F7B7FBF1FCBA
:1030D000642710FB07F7B7FBF1F7CDE90621CDE92F
:1030E000041CCDE902700D4A08213046CDE9008963
:1030F00000F0A4FA641CAC42D4D308B0BDE8F08759
:1031000042616420617267756D656E7420636F75CE
:103110006E740000A06A0000686A00000C63000082
:1031200070B515468268D2F83C41C4F3400424B11E
:103130001A46294600F0AAFA06E039B1516804A2FD
:103140000B68022100F07AFA012070BD002070BDEA
:1031500025733A2077726F6E6720706172616D65BA
:1031600074657220636F756E740D0A0010B50446A5
:1031700002290CD1A068D0F83C01C0F3400030B166
:1031800020460022BDE81040114600F07FBA064AF2
:1031900006A1206900F036FD034A2069BDE8104011
:1031A000093202A100F02EBDF05F0000257300007F
:1031B000012907D0022909D18168D1F83C11C1F356
:1031C000400119B10022114600F060BA01A20221AB
:1031D00000F034BA506C6561736520737065636983
:1031E0006679206120737562636F6D6D616E642E08
:1031F0000D0A00001CB5012905D002290BD014D9F5
:103200004FF0010112E002B04FF00002BDE81040A3
:10321000114600F03BBA536808A1CDE900131368CA
:103220000CA2022100F00AFA1CBD002102B000230A
:10323000BDE810401A46FFF773BF000020756E6BA3
:103240006E6F776E20706172616D657465723A2081
:103250000000000025733A257325730D0A00000055
:1032600010B50446012901D0012100E0002100230E
:103270001A46FFF755FF002808D1A168C1F82C01B4
:10328000E068C068BDE8104001F090BA10BD0000D1
:103290003EB50446012901D0012100E000210023B0
:1032A0001A46FFF73DFF002818D1E068C06801F01A
:1032B0007AFAC0B2642110FB01F2E168C96889683A
:1032C000B2FBF1F2D2B20092CDE90101A06804A2F2
:1032D0000821D0F82C31204600F0B0F93EBD0000A6
:1032E0004C6F7374206C6F67733A2025750D0A4D0F
:1032F0006178206C6F6720717565756520757469DC
:103300006C697A6174696F6E3A2025752525205B9A
:1033100025752F25755D0D0A000000007CB514464B
:103320000546012903D0022908D0012107E002B097
:103330000022BDE87040114600F0A8B9002100232A
:103340001A46FFF7EDFE002809D1616804A0CDE917
:10335000000109A202212846236800F06FF97CBD14
:1033600020756E6B6E6F776E20706172616D657423
:1033700065723A200000000025733A257325730D0D
:103380000A00000010B50446012901D0012100E027
:10339000002100231A46FFF7C3FE002806D1A068CB
:1033A000D0F83C1121F00401C0F83C1110BD10B55B
:1033B0000446012901D0012100E0002100231A4622
:1033C000FFF7AEFE002806D1A068D0F83C1141F00E
:1033D0000401C0F83C1110BD7CB514460D460646EC
:1033E000022901D9012100E0002100231A46FFF73C
:1033F00097FE002811D1022D05D03046FDF716FEAC
:1034000060B10BA30BE061680AA0CDE900010FA237
:1034100002213046236800F011F97CBD0EA302B0F2
:103420003046BDE870400DA2082100F007B9000049
:103430006F6E000020756E6B6E6F776E207061721C
:10344000616D657465723A200000000025733A25AD
:103450007325730D0A0000006F6666004563686F90
:10346000207374617475733A2025730D0A0000008F
:1034700010B50446012901D0012100E000210023FC
:103480001A46FFF74DFE002806D1A068D0F83C117F
:1034900021F00801C0F83C1110BD10B50446012907
:1034A00001D0012100E0002100231A46FFF738FE79
:1034B000002806D1A068D0F83C1141F00801C0F8FE
:1034C0003C1110BD7FB50446012901D0012100E067
:1034D000002100231A46FFF723FE002827D1A06809
:1034E0000026D0F83451F5B101E0082E1BD200239C
:1034F000092201A9284601F0BCF89DF80C20A1681A
:10350000092328469431521C01F0B3F8A0683346D1
:1035100094300090029D761C05A20821204600F000
:103520008DF8002DE1D1A168002081F894007FBDC5
:103530005B2533645D2025730D0A00007CB51546BC
:103540000446012903D0022917D9012116E0A168F8
:1035500001F10C020D3102F07BF800281ED0A168A9
:1035600050200FA24873A1681820087302B02046AB
:10357000BDE87040042100F061B8002100231A4624
:10358000FFF7CEFD002809D1696814A0CDE900013C
:1035900018A2022120462B6800F050F87CBD0000E4
:1035A0004E6F20726573706F6E73652066726F6DFB
:1035B00020746865207465726D696E616C2C206181
:1035C0007373756D6564203830783234207363729C
:1035D00065656E2073697A650D0A000020756E6B53
:1035E0006E6F776E20706172616D657465723A20DE
:1035F0000000000025733A257325730D0A000000B2
:1036000010B50446012901D0012100E0002100236A
:103610001A46FFF785FD00280AD1064A06A120694F
:1036200000F0F0FAA16850204873A16818200873D0
:1036300010BD000006600000257300000FB438B50F
:10364000044607A80090A068D0F83C21520717D57F
:10365000C27B8A4214D0B0F80F50204602F040FBE3
:103660006A462069069900F0E6FAE9B2204602F0BF
:1036700037FB290A204602F015FB38BC5DF814FB25
:103680006A462069069900F0D6FAF6E72DE9F04F70
:10369000804689B016460C468948FDF78DFE0546E2
:1036A00087483338FDF788FE281A1FFA80F98448C6
:1036B00084A220380090D8F80800082140680368E8
:1036C0004046FFF7BBFFD8F8080040680068FDF7E8
:1036D00073FE05467A482038FDF76EFE284482B214
:1036E000D8F808000023406841684046FEF74EFDC8
:1036F00076A208214046FFF7A1FF16B30CB30025C0
:103700001DE000BF05EB450A04EB8A0BDBF8040063
:10371000FDF752FE074654F82A00FDF74DFE391812
:1037200049450BD9DBF80400FDF746FE074654F87F
:103730002A00FDF741FE38441FFA80F96D1CB5429E
:10374000E0D35F483338FDF737FE4844801C1FFA4A
:1037500080F95B4800904B465FA208214046FFF786
:103760006DFF09F1030087B2079000233A465CA180
:103770004046FEF70BFD002C52D000254EE000BF66
:1037800005EB450A04EB8A0B54F82A00DBF80430F9
:103790006BB350B34A4957A23339CDE90010082121
:1037A0004046FFF74BFF09F102000090DBF80400F0
:1037B000FDF702FE074654F82A00FDF7FDFD074419
:1037C0003F483338FDF7F8FD39180098401A801E3D
:1037D000C1B24046FEF7F8FA3A224949D8F810003B
:1037E00000F010FA0098401C0AE0009301E040B19C
:1037F00000904B4638A208214046FFF71FFF07986C
:1038000087B2DBF8081029B100233A464046FEF79C
:10381000BDFC02E04046FEF705FA6D1CB542AFD391
:10382000D8F8080040688068002845D0814600200C
:103830000446064603AD02903246761C02AB0121D7
:1038400048460095FEF73EF8029850B10068FDF733
:10385000B3FDA042F0D902980068FDF7ADFD84B237
:10386000EAE7012E28D027A208214046FFF7E6FE0E
:1038700000273A467F1C02AB012148460095FEF71F
:1038800021F80298002817D0A11C8EB20068009081
:10389000334611A208214046FFF7D0FE0298F61CDD
:1038A000B2B2416821B100234046FEF76FFCE0E769
:1038B0004046FEF7B7F9DCE709B0BDE8F08F00003D
:1038C0000C60000025732573000000004F707469C0
:1038D0006F6E733A0D0A00002020252D2A733A00DE
:1038E00053686F7720636F6D6D616E642068656CDF
:1038F000702E000020202573257325730000000022
:10390000F80D0000537562636F6D6D616E64733AFC
:103910000D0A00002DE9F0411E460546069F00F005
:1039200011F804000CD15EB13946E86800F00AFBDA
:10393000002802DA0420BDE8F081E8680121417224
:103940002046F8E770B50446C06815462346446132
:10395000606802681668264AB047002846D1606948
:1039600000F076FE002841D1A168C1F83001A168BD
:10397000C1F834014FF4A071A068FCF748FDA068BD
:10398000D0F83C1141F02001C0F83C11A068D0F8FB
:103990003C1165F38201C0F83C11A068D0F83C11DD
:1039A00041F00801C0F83C11A1680120124B0870D9
:1039B000A1685020114A4873A1681820087300219B
:1039C0000C48D21A07E000BF03EBC1046468246806
:1039D00040F82140491CB1EBD20FF5D3072A04D996
:1039E000D108074B0422FCF79DFC002070BD0000AD
:1039F000D5160000FC000020D0690000106A00000D
:103A0000495600000023FDF70FBF000010B5044623
:103A10008068102100F59E70FFF7C5FAA068007855
:103A2000F8B101281DD002281BD12046FDF7BFFBAD
:103A300000212046FDF700FB98B110A2032120468B
:103A40002368FFF7FBFD2046FDF7F0FA48B1A368B5
:103A50000AA2082120461433FFF7F0FD2046FEF7A6
:103A60007DF9206900F0DBF8A068BDE810406FF038
:103A7000100100F59E70FFF781BA00002573000069
:103A800070B5044680680078012801D0082070BD18
:103A9000606801688A680021904705000FD10821FD
:103AA000204602F01DF90121204602F0FBF805A195
:103AB000206900F0A7F802212046FDF769FC28469E
:103AC00070BD00000D0A0A0000F180400068002867
:103AD00000D00120704708B500F18040002101604E
:103AE0000068009008BD000070B50A4C207808B14D
:103AF00085250CE00020A06060602061E060064841
:103B000001F086F8054601F06DF801202070284686
:103B100070BD00005C050020A918000070B5104DB4
:103B20000446A87838B114B16168012088470020A4
:103B3000FCF734FF0CE00020FCF730FF24B108480C
:103B400021461030FEF7BEFDE86808B901F070F8B4
:103B5000E868401CE860BDE870400020FCF720BF2A
:103B60005C050020F0B505460478154889B0164676
:103B700040F82420124A08690832A2F10C0742F8E2
:103B80002400487F385520226846FCF719FC04942D
:103B90002878385C48B10EB10A4A00E00022694634
:103BA000281D01F03DFA09B0F0BD0EB1064A00E053
:103BB0000022694605F10C0001F084F8F3E70000EB
:103BC000440000209D5A00004559000030B403789D
:103BD000054CE35C1BB130BC001D01F0DDBA30BC0C
:103BE0000C3001F059B90000400000200178044A6F
:103BF000515C11B1001D01F025BB0C3001F0AEB9D4
:103C0000400000200FB408B50399002904D004AA8D
:103C100000926A4600F00FF801B05DF814FB10B591
:103C200082680446002A05D0D4E904032168984735
:103C30000020A06010BD2DE9FC4791460C00804695
:103C400076D014F8011B39B125290ED04046FCF777
:103C500075FF20780028F4D198F80C00002867D070
:103C60004046BDE8FC47FFF7DABF0020012221787B
:103C70002B291BD02D2902D0302908D102E040F099
:103C8000010001E040F00200641C002AEFD1002591
:103C90002A290ED02178A1F130020A2A11D205EB8F
:103CA000850201EB4205641C303DF1E740F0040061
:103CB000EAE7D9F800100B1DC9F800300968641C48
:103CC0000D44217800232E290BD114F8011FA1F1F6
:103CD00030020A2A05D203EB830201EB4203303B98
:103CE000F3E76C290DD068290BD0692921D00BDCB2
:103CF000252918D0582931D063290ED0642915D12F
:103D000017E014F8011FECE7702969D0732932D04D
:103D100075291BD0782909D120E0D9F80000011DB0
:103D2000C9F8001001784046FCF708FF641C90E7D2
:103D30006CE0D9F800100A1DC9F800200968CDE927
:103D400000500A224046FEF703FCEFE7D9F80010C6
:103D50000A1DC9F8002009680A2206E0D9F80010F7
:103D60000A1DC9F8002009681022CDE9005040461C
:103D700001F026FFDAE7D9F8001000270A1DC9F87C
:103D800000200E68C00705D112E04046761C7F1C5B
:103D9000FCF7D4FE31780029F7D104E02021404619
:103DA0006D1EFCF7CBFEBD42C0D9002DF6D1BDE79C
:103DB0004EB13046FCF736FB074604E02021404672
:103DC0006D1EFCF7BBFEBD4206D9002DF6D103E007
:103DD0004046761CFCF7B2FE31780029F8D1A5E701
:103DE000D9F80000011DC9F80010056830214046CF
:103DF000FCF7A4FE78214046FCF7A0FE0820002135
:103E0000CDE90001034610222946B0E7BDE8FC8752
:103E10002DE9FF411C46DDE90A7815460E46684645
:103E200000F060F846EA450141EA840141EA0722D0
:103E300042EA0841009A00EB8200C0F80017BDE892
:103E4000FF812DE9FF411C46DDE90A7815460E4643
:103E5000684600F055F846EA450141EA840141EA26
:103E6000072242EA0841009A00EB8200C0F80017DE
:103E7000BDE8FF811CB5002100910B460122019194
:103E8000FFF7C6FF1CBD1CB5002100910B460122A7
:103E90000191FFF7D6FF1CBD1CB500220B46009216
:103EA00011460192FFF7B4FF1CBD1CB500220B4662
:103EB000009211460192FFF7C4FF1CBD1CB5002102
:103EC00000910B46012201911146FFF7A1FF1CBD95
:103ED0001CB5002100910B46012201911146FFF70C
:103EE000B0FF1CBD0168202902D24FF0A0407047EE
:103EF00001F01F01016001487047000000030050FD
:103F00000168202902D24FF0A040704701F01F0144
:103F100001600148704700000003005001B5684689
:103F2000FFF7E0FF009A01219140C0F8081508BD95
:103F300001B56846FFF7E4FF009A01219140C0F8FF
:103F4000081508BD2DE9F0410E461C490446002520
:103F5000D1F81024104609E0037AAB4205D16D1C5C
:103F60000A2DF7DB4FF0FF3525E040680028F3D13C
:103F7000681C20D02572D1F8100440B14068606000
:103F8000D1F8100444600027DFF834800FE00020EF
:103F9000C1F810446060F6E708EBC700C279B2428E
:103FA00000D33246207A394600F066FA7F1C00F0D2
:103FB00033FAB842F0D82846BDE8F0818C070020DB
:103FC000106A000038B54469C0680022694600F0F4
:103FD0008EFB002803D100212046FDF72DF838BDC7
:103FE00010B54469606801688A680121904718B17A
:103FF0000420A168087010BD0320FAE72DE9F34101
:1040000046690446B068007804281ED0032807D00B
:10401000002501A9E06800F0D4FB85F0010709E064
:104020000125F6E739463046FDF706F801A9E068B4
:1040300000F0C7FB0028F5D1019800F005FB002D2A
:1040400003D000213046FCF7F7FFBDE8FC810000FB
:104050000A4A012902EBC00007D0022907D0032930
:1040600007D0042907D000207047022070470420A1
:10407000704700797047407970470000106A00006F
:104080002DE9FF5FFCF76AFD18B1002004B0BDE820
:10409000F09F874C0020C4F81804BFF34F8F60686E
:1040A0000090A6684FF00009304004EB800008E063
:1040B00021680098814201D86160E6E7304004EB56
:1040C00080000C306946FEF7D7FA0028F0D101AA2B
:1040D000A046009901EA060408EB8403491CDB684A
:1040E00042F82030401C00910228F2D3019800F0E1
:1040F0000300022802D0012850D0BEE001985022CF
:10410000810D8A46B2EB905F00D850210C4664F3D3
:104110009F50C0F3C20701900831664800F04BFA87
:104120000500EAD000F090FA4B46082201A9284683
:1041300000F0A5FA009909F1080B3140701A8000CF
:10414000001D844223D95A4E0C3630B1C2B208EB5E
:104150008101201A91460C3104E03146E2B200267A
:1041600091463046C4B25B46284600F088FA0BEB15
:1041700009032EB1224631464FEA050000F07FFACE
:1041800000990AF1030001EB900000903DE008EB7C
:1041900081015B46224628460C31EFE70198C0F3C7
:1041A0008310062800D30620019960F38911C1F31A
:1041B0008310C1F3C207801C019181003D4800F0CB
:1041C000FAF9050059D000F03FFA4B46082201A940
:1041D000284600F054FA09F1080900240FE000987D
:1041E0004B460246304008EB8001501C00900422F0
:1041F00028460C3100F043FA09F10409641C0198C7
:10420000C0F38310A042EAD8B5B3D8F81044D8F868
:1042100018044646F8B1284600F01CFA42E0607ADD
:10422000012817D1BDF80800234A00EB400002EB3B
:104230008000217A806801EB4101C84000F007004E
:10424000052F00D10327B84204D32268204629460F
:10425000126890476468002CE1D1284600F0FAF912
:104260000020FCF79BFBD6F8180408B90098706092
:104270000020FCF795FB15E0FFE7D8F8104404E0B8
:1042800021682046896888476468002CF8D10B486B
:104290004168022906D30088022101EB004008A1F1
:1042A00000F018F8FCF75AFC80F00100EEE6000080
:1042B0008C070020846A00001C010020940100206B
:1042C0004261636B656E647320666C7573686564C8
:1042D0000000000000231A4601F070B92DE9F047F4
:1042E0000E4680461C46924608293ED894F80C900B
:1042F000002020731946104601F062F80025B542EF
:1043000006D218F805201AA12046FFF77BFC03E02F
:1043100019A12046FFF776FC6D1C082DEFD317A1DD
:104320002046FFF76FFC0025B54210D218F8057043
:10433000FBF7F4FF0068C05D10F03E0F01D03A4675
:1043400000E02E220EA12046FFF75CFC03E00DA149
:104350002046FFF757FC6D1C082DE5D301222146AE
:10436000504601F00FF884F80C90BDE8F08700008B
:104370002025303278000000202020007C00000042
:1043800025630000200000002DE9F0471D484FF094
:104390000009FF21C0F80090C0E90191C0F818940D
:1043A000C0F8149480F82094174800F051F90028C0
:1043B00026D11649DFF85880A1EB0800C708002471
:1043C0001BE0002635460CE0AC4209D058F834001A
:1043D00058F835101422FCF743F8002800DD761C4D
:1043E0006D1CBD42F0D30B4904EB440001EB80008F
:1043F000C0F8049004804680641CBC42E1D30020D5
:10440000BDE8F0878C070020846A0000686A00001D
:10441000106A00001C01002002480349401AC0082D
:1044200070470000686A0000106A00007FB505460A
:104430001146002401A87BB1FEF73EFDA0B901980A
:104440000B4900EB400001EB800005EB4501806863
:10445000C84000F0070407E0FEF72EFD20B905482C
:10446000019900EBC100847904B0204670BD0000C2
:104470001C010020106A000030B50F4B01EB410118
:1044800003EB810400EB40000723A56803FA00F169
:104490008D4302F007018140294300252A46A1608F
:1044A00003FA02F00840D040A84200D90546D21CC9
:1044B0000A2AF5D3656030BD1C01002013B568469B
:1044C000FEF7FAFC08B100201CBD0248009950F824
:1044D00031001CBD106A000070B508480125D0F8F5
:1044E000104480F8205405E0657221682046496830
:1044F00088476468002CF7D170BD00008C0700204D
:104500002DE9FF4781460C9D00200C462F7B287328
:10451000984616462946184600F052FF072E42D20A
:10452000DFE806F004090F161F2A36004946284620
:10453000FFF768FB37E0494628462268FFF762FB31
:1045400031E0D4E9002349462846FFF75BFB2AE027
:10455000A0680090D4E9002349462846FFF752FBA3
:1045600021E0D4E90201CDE90001D4E90023494664
:104570002846FFF747FB16E004F1080007C88DE85E
:104580000700D4E9002349462846FFF73BFB0AE031
:1045900004F108000FC88DE80F00D4E90023494654
:1045A0002846FFF72FFB00222946404600F0EAFE8E
:1045B0002F73BDE8FF872DE9F041058B80462D1F45
:1045C0004819C01CB0FBF5F0C6B24046FEF7F7FC38
:1045D000041E19D00020207101206071E5800027A1
:1045E0002546761EC4F800800BE04046FEF7E7FC47
:1045F00060B16179491C6171286005467F1CC0F873
:104600000080B742F1D32046BDE8F081204600F09B
:1046100002F80020F8E72DE9F041457901466B1ECC
:10462000002201E00968521C9A42FBD30F68014640
:10463000002605E038460C68FEF7E0FC2146761CB3
:10464000AE42F7D3BDE8F0810121001DFEF790BC1A
:10465000FEF7E9BC10B504460121001DFEF7A9FCD8
:1046600010F0FF0F04D12046BDE81040FFF7D3BF84
:1046700010BD38B501240094FEF7CFFB38BD38B526
:1046800000240094FEF7C9FB38BD0000094902224E
:104690000A60BFF36F8FBFF34F8F0A1D106006488B
:1046A0000268002AFCD000200860BFF36F8FBFF3C0
:1046B0004F8F704704E5014000E40140094A01239F
:1046C0001360BFF36F8FBFF34F8F0160064801681F
:1046D0000029FCD000201060BFF36F8FBFF34F8F15
:1046E0007047000004E5014000E4014070472DE9F7
:1046F000F0410446002790460E463846FCF74EF936
:10470000204600F038F830B105270020FCF748F9C2
:104710003846BDE8F08120680568B8F1000F05D182
:104720000168204600F046F821680860E268012A26
:104730000CD0022A0ED0042A11D06068082A13D0A7
:1047400005FB02013046FBF73BFEDEE76068405D9B
:104750003070DAE7606830F815003080D5E76068BF
:1047600050F825003060D0E700EBC500D0E900101C
:10477000C6E90010C9E7016808684968884201D1A4
:10478000012070470020704701680A684968806806
:10479000884201D9491C00E00021914201D1012049
:1047A00070470020704700688068704700680021EB
:1047B000816070478068884201D9481C704700209A
:1047C00070472DE9F04104464FF000080E46404680
:1047D000FCF7E4F82046FFF7D7FF070009D0207C5C
:1047E00038B14FF004080020FCF7DAF84046BDE885
:1047F000F0812068456841682046FFF7DBFF2168AB
:10480000486037B1206801682046FFF7D3FF216870
:104810000860E268012A14D0022A16D0042A19D0AE
:10482000082A1CD06068314605FB0200FBF7C8FD72
:10483000204600F01DFE21688A688242D3D288603B
:10484000D1E7616830784855F2E76168308821F82F
:104850001500EDE76168306841F82500E8E7D6E922
:104860000001626802EBC502C2E90001E0E7000056
:104870002DE9F04F8146806889B0D0F83C01C0F343
:10488000400038B109B04846BDE8F04F002211465B
:10489000FEF7FCBE012907D909B04846BDE8F04F34
:1048A0001DA20221FEF7CABE2049DFF884B0A1EBA9
:1048B0000B001C21B0FBF1F8002526E0C5EBC5017B
:1048C0000BEB81042068D4E9026A8768204600F077
:1048D0003FF86421794364224243B1FBF6F1B2FB15
:1048E000F6F26369247CACB112A400BFCDE9066482
:1048F000CDF800A00597CDE90120CDE90361104A6C
:1049000008214846FEF79AFE6D1C4545D6D309B0EE
:10491000BDE8F08F0BA4E9E742616420617267751E
:104920006D656E7420636F756E740000BC6A000064
:10493000A06A00004E6F206F766572666C6F77001C
:10494000806600004F766572666C6F77000000002D
:1049500010B504460020FCF721F8204600F088FD41
:1049600004460020FCF71CF8204610BD2DE9F0415C
:104970001E0015460F46044606D0A068FEF7F5FA5D
:1049800010B11120BDE8F081A0686268D0E9033160
:10499000A3EB010C501C844507D10020286016B100
:1049A000A068FEF7D9FA0020ECE703EA020001EA6A
:1049B0000206B04202D3111A491C00E0C91A2A6843
:1049C0008A4200D211462960216808443860A068F4
:1049D0002A68C1681144C160E5E72DE9F041054648
:1049E000806817468846001DFEF7BFFA10B11120F7
:1049F000BDE8F081A868816800690C1A3868A04297
:104A000000D204463C60AA68696810699268084050
:104A10000A40824201D9161A01E00E1A761CB442ED
:104A200008D92968324608444146FBF7C9FCA41B53
:104A30000020B0442968224601444046FBF7C0FCF0
:104A4000A8683A68016911440161A868001DFEF771
:104A500083FA0020CCE72DE9F04105461746884649
:104A60008068FEF782FA10B11120BDE8F081A868D5
:104A700081680069081A69680C1A3868641CA042C9
:104A800000D204463C60A8686968806808400E1A35
:104A9000761CB44208D92968324608444146FBF7DF
:104AA0008FFCA41B0020B0442968224608444146DC
:104AB000FBF786FCA8683A68816811448160A868A1
:104AC000FEF74AFA0020D0E710B5826894681369AF
:104AD000E41AA14201D9042010BD19441161826871
:104AE00051618068001DFEF737FA002010BD2DE9E6
:104AF000F0411E0014460F46054607D0A868001D69
:104B0000FEF733FA10B11120BDE8F081A868816882
:104B100040690A1A09D06B681840194081420DD9C2
:104B2000266896420AD9226010E0002020601EB15B
:104B3000A868001DFEF710FA0020E5E7814205D8BD
:104B4000191A2268491C8A4200D921602968084440
:104B50003860A8682268416911444161ECE78268C5
:104B60000021916082681161826851618268D16020
:104B70008268516080680160704770B582684568DE
:104B800094681369E31AEB1A5B1C994201D904205B
:104B900070BD214491608268D1608068FEF7DFF9C2
:104BA00008B1002070BD082070BD4058002800D01A
:104BB0000120704708B5002242504058009008BDBF
:104BC000D0F80403084000D0012070474058002866
:104BD00000D00120704708B5002242504058009094
:104BE00008BD000008480068012110F0010F08D13D
:104BF0004FF0E020E02280F80024C0F88012C0F8D6
:104C0000001102480160704700E100E01805004013
:104C10000649024600200B790BB1852070470A60D7
:104C200001220A7100224A717047000054000020DE
:104C300010B54FF48270FEF74EFF02204107C1F815
:104C4000040302490120086010BD00000800004074
:104C5000002802D00149800108477047215E00000A
:104C60000121B1EB507F01D1012070470020704736
:104C700070B50D4600F0F0FB04000FD00020FBF7EC
:104C80008DFE207920B10020FBF78AFE112070BD37
:104C90000120256020710020FBF782FE002070BDFE
:104CA00010B500F0D9FB002802D00021016001718D
:104CB00010BD00000149024800F05CBE70050020F4
:104CC000002000402DE9F0410546007916460F46C8
:104CD00000EB40012D4A01EBC00102EB810494F886
:104CE0002A1011B10820BDE8F081294951F820109F
:104CF0002868FFF7BDFF08B11120F4E739462846C0
:104D0000FBF762FE66603869206030004FF00106F4
:104D10002FD03F7F4FF48E712868FFF74BFF4FF481
:104D2000A2712868FFF746FF28681A49C0F80413E3
:104D300028684FEA4711000B40B2002806DA00F05D
:104D40000F0000F1E02080F8141D03E000F1E020E6
:104D500080F800142868000B40B200F01F0206FA29
:104D600002F14009800000F1E020C0F88012C0F894
:104D7000001128680421C0F800150020A061E0613E
:104D800084F8290044F8140FA675ACE770050020DC
:104D90000C5E0000800002002DE9F05F05460079FE
:104DA0004FF4017600EB400303EBC000344B03EB00
:104DB00080040020636813B12B68C3F80863A369FB
:104DC0004FF000096BB1E06938B1606810B1286834
:104DD000C0F804631120BDE8F09FE2610120216169
:104DE00005E0C4F82490A261E160C4F81C9094F836
:104DF0002910014302D1284600F094FB6068002886
:104E0000286803D0C0F804630020E4E74FF4A276DA
:104E10003146FFF7CFFEB2464FF4927B59462868E1
:104E2000FFF7C3FE06464FF484712868FFF7BDFE06
:104E3000804651462868FFF7B8FE074648EA070053
:104E40003043EBD056EA070007D12146286800F02E
:104E500039FBA169606A8142E0D8C4F818900EB1AC
:104E60000320B8E70FB10F20B5E794F8291001200F
:104E70000029296801D00860C6E74860C4E700003F
:104E80007005002001684FF40172C1F80823006822
:104E900001214160704700002DE9F0470546007987
:104EA0000B4600EB400101EBC000234901EB8004FD
:104EB000284600F043F810B11120BDE8F0874FF00C
:104EC0000008C4F82080A360626184F828804FF451
:104ED0008E76474631462868FFF76CFE28684FF00B
:104EE0000109C0F808902146286800F0D7FC6068E6
:104EF00000BBD5F800A00EE094F8280008B10F27F9
:104F000016E031465046FFF750FE0028F4D0214607
:104F1000504600F0C3FC216A60698142F1D33146FA
:104F20002868FFF742FE0028F9D02868C0F80C90E6
:104F3000C4F814803846C0E770050020007900EB03
:104F4000400101EBC000044901EB800040690028EA
:104F500000D0012070470000700500202DE9F047C7
:104F6000044600794FF0000900EB400101EBC0005E
:104F7000254901EB80072068C0F80095786880B16A
:104F800020682249C0F8081320680121000B40B2B4
:104F900000F01F0291404009800000F1E020C0F8BD
:104FA00080112068D0F80C25D0F81485D0F8086559
:104FB000D0F810554FF0FF31C0F81415C0F80C159B
:104FC0002068C0F80815C0F81015501C02D0104613
:104FD000FEF750FFB8F1FF3F02D04046FEF74AFF10
:104FE000681C02D02846FEF745FF701C02D03046F0
:104FF000FEF740FF2068FFF753FE87F82A90C7F8B6
:105000000490BDE8F08700007005002084020200D3
:105010000149024800F05ABD9C05002000200040D4
:105020002DE9F0410546164600790F46154A00EB7A
:10503000C00102EB810494F8201011B10820BDE8F2
:10504000F081114951F820102868FFF711FE08B1CE
:105050001120F4E739462846FBF7F1FC6660386911
:1050600020601EB1397F2846FDF7C6FA286808215E
:10507000C0F800150020A061E0610121606184F8A2
:105080002010DCE79C050020105E00002DE9F05F99
:10509000044600790E4600EBC001DFF8F0A0174689
:1050A0000AEB81053046FFF7DBFDB0B168684FF0D1
:1050B00000084FF4047910B12168C1F80893A86979
:1050C0004FF0000B80B1E86948B1686810B1206802
:1050D000C0F804931120BDE8F09F1020FBE7EF61BA
:1050E0004FF001082E6102E0EE60C5E9067B002565
:1050F0004FF488712068FFF76EFD4FF4A2712068AD
:10510000FFF769FD2068C0F83465C0F8387520687D
:10511000B8F1000F12D0D0F8001241F02001C0F811
:1051200000122079D04600EBC0010AEB81004068F4
:1051300038B12068C0F804932846CCE7012101600B
:10514000EFE74FF4887A4FF4A27951462068FFF7D1
:105150003DFD074649462068FFF738FD06464FF4F7
:1051600092712068FFF732FD014647EA06000843C6
:10517000EBD0227902EBC20308EB8302C2F818B02D
:1051800001B10325002ED7D00F25D5E79C050020BF
:1051900000680121416070472DE9F04704460E4642
:1051A0000079204900EBC00001EB8005174630462E
:1051B000FFF756FD30B1204600F036F820B111203F
:1051C000BDE8F0871020FBE76F61AE604FF490768A
:1051D000002731462068FFF7FEFC4FF4AC784146CB
:1051E0002068FFF7F8FC2068AA686969C0F84425C0
:1051F000C0F84815206801218160686878B9B14617
:1052000049462068FFF7E2FC064641462068FFF762
:10521000DDFC0643F4D000B10F270020686138465A
:10522000CEE700009C0500200079054900EBC00096
:1052300001EB80004069002800D001207047000089
:105240009C0500202DE9F04704460079274900EB32
:10525000C00001EB800720684FF00009C0F80095FE
:10526000786880B120682249C0F8081320680121BD
:10527000000B40B200F01F0291404009800000F195
:10528000E020C0F880112068D0F80C25D0F81485F3
:10529000D0F80865D0F810554FF0FF31C0F80C1564
:1052A000C0F814152068C0F80815C0F81015501C77
:1052B00002D01046FEF7E7FDB8F1FF3F02D04046AE
:1052C000FEF7E1FD681C02D02846FEF7DCFD701CED
:1052D00002D03046FEF7D7FD2068FFF7E1FC87F8E3
:1052E0002090C7F80490BDE8F08700009C050020DE
:1052F000100302002DE9F84317460C0005462BD099
:10530000DFF870804646D8F80000FCF755F83844BE
:10531000C7B23068FCF750F8A968497B081AB0FB9F
:10532000F7F0C6B22046FCF747F8A968381AC7B2AA
:10533000487CB0FBF6F206FB1202401C487482B1B6
:1053400023460DA207212846FEF778F9394628465C
:10535000BDE8F843FCF738BDA96800204874BDE8F3
:10536000F883009405A207212846D8F80030FEF7FC
:1053700065F9EBE77C000020257300000D0A25731A
:105380002573000010B50C46017A052908D0407A33
:1053900038B1084808A102682046FEF733FC00E057
:1053A0001AB106A12046FEF72DFC2046BDE81040AC
:1053B000FEF735BCD4000020257300000D0A000064
:1053C00038B5C3880D46044633B114A0009015A229
:1053D00016A12846FEF716FC217A05291CD0607A12
:1053E00048B1A088FEF734FE164951F8202016A1D6
:1053F0002846FEF707FCA0880021FFF75FF8034668
:105400001049207A143951F8202001B02846BDE80F
:1054100030400EA1FEF7F6BB38BD00001B5B306DBF
:10542000000000001B5B313B33316D0025734C6F76
:1054300067732064726F7070656420282564292565
:10544000730D0A00D4000020257300003C25733E34
:105450002025733A200000000349884201D1034807
:105460007047002070470000002000405C000020D2
:1054700001680A684968914201D3881A70478068B8
:10548000801A0844401C704770B5012670044FF024
:10549000E0210025C1F88001084C4010C4F8480301
:1054A000C4F8080366602F20FFF7D2FBA660044C07
:1054B0002F20A560FFF7CCFBA57070BD0010014048
:1054C0006400002070B5054688690C4600284FF43A
:1054D000847128460AD0FFF76DFBD5F81805626A7B
:1054E000E1688854606A401C606270BDFFF762FB2F
:1054F000D5F8180570BD1FB501238DF80030CDE932
:105500000121D0E90012684690471FBD1FB5012355
:105510008DF800308DF808100192D0E9001268462D
:1055200090471FBD10B5044600684FF49271FFF715
:1055300041FB4FF484712068FFF73CFB2068012198
:10554000016010BD7CB50446FF20009001236A462F
:1055500001A9E068FFF70AFA002819D1009A002A89
:1055600016D060690B4D01990378D2B2EB5C1BB188
:10557000001DFFF78BFD02E00C30FFF70DFC00284B
:1055800006D1A068224640F6CD410068FBF7B6F987
:105590007CBD0000400000200022CA604A60054A2D
:1055A0008A60052803D2044A52F8200000E0002057
:1055B0000860704774600000940000202DE9F84FE7
:1055C000204D92468946064698460122694618466D
:1055D000AF68FBF76FFA58B3009800210446801CAF
:1055E00009E000BF00EA07035AF8212005EB830316
:1055F000401C491CDA604145F4D34FEA164AFCF7D7
:10560000FBFB4AEA0041601C384005EB80003C404F
:1056100005EB8402C160D06866F3C50068F38910A9
:1056200069F39F2020F00300401C20F00400D060AC
:1056300095F8200402E000BFFEF722FD0028FBD110
:10564000BDE8F88F8C07002009680068FAF7F1BE02
:105650002DE9F04115460E460446FCF7EDFA78B9FF
:10566000A068FA21077A90F80A802046FCF7ACFB84
:10567000FA212046FCF758FA2046FCF7DDFA10B173
:105680000620BDE8F081A068007A3070A068807ABA
:1056900028703078C01BC1B22046FCF7B7FA2978D1
:1056A000A1EB0800C1B22046FCF79AFB0020E8E716
:1056B0004069054A0178515C11B1001DFFF768BDD2
:1056C0000C30FFF7DFBB0000400000202DE9F84F51
:1056D0001D4C00256846D4E901A6FCF797FB00277E
:1056E00038B30023009A61681CE0D1F800C0084676
:1056F000944503D9ACEB02020A6015E0A2EB0C0260
:1057000063440760D0F80CC0C1698146BCF1000F4A
:1057100008D006EB030828F07F48C0E9018CC9F8DF
:105720001C5005460029E0D128466160FCF7D6FFF1
:1057300003E02846FCF7D2FF10B15046FCF754F9BD
:10574000E770BDE8F88F0000640000200D4B10B535
:10575000596831B102680C68A24204D8A21A0A60E2
:10576000C161586010BD0B4603E00B46C969121BAE
:1057700021B10C689442F8D3A41A0C600260C16194
:10578000D86110BD640000202DE9F041144E776807
:105790003D462C4603E0844204D02546E469002CB3
:1057A000F9D11BE0D4B1A5420BD1F869706040B9C2
:1057B0000C49012088600021B160F0702F20FFF7B4
:1057C00047FA2168E069E86110B10268114401609C
:1057D0007068874202D00120BDE8F0810020FBE71D
:1057E0006400002000100140F8B5064600240D4674
:1057F0002046FBF7D3F8684600F03CFA68B1057024
:10580000084946609DF8000048700020FBF7C8F882
:105810001420FAF788FE2046F8BD04240020FBF788
:10582000BFF8F8E7C00500202DE9F041194D6C687C
:10583000002C2CD0184800270068A968B846401AE8
:1058400020F07F462068B0420CD82146361A074423
:10585000E469087C20B181F810808869496988472B
:10586000002CEFD129786878814206D1401CC0B263
:105870006870022801D185F80180064869780C30EB
:1058800040F82170BDE8F0411420FAF74CBEBDE8A5
:10589000F0810000640000200415014070B50C4642
:1058A00005464FF48E71FFF785F9216AA068415CC7
:1058B000206A401C2062C5F81C1570BD1FB500226F
:1058C0008DF800200291816801914261D0E90012B7
:1058D000684690471FBD7CB5FF26054600960078B8
:1058E0000C46B8B1012806D0022812D1297AE06806
:1058F000FFF743F90AE0297AE068FFF73EF9287AD2
:1059000020B16068D0E90021002090472046FFF7D1
:1059100019FE7CBD297A2069FFF7D6F8009601238D
:105920006A4601A92069FFF7E2F8009820B1C2B2E7
:1059300060690199FEF74AF96068D0E90021012009
:1059400090477CBD1FB50A4601788DF8001041686C
:105950000191017A8DF80810C0680390044850F84E
:105960002210083850F82220684690471FBD0000DA
:105970004C0000202DE9FF470C4605464FF400710E
:10598000FFF71EF901274FF40178002618B34FF4F2
:10599000927949462846FFF708F9E0B1494628467A
:1059A000FFF708F9C5F8088394F8290000B96F607B
:1059B00002208DF80000D5F88004C5F8800403901B
:1059C000A0690290E0680190A661E661D4E9001246
:1059D0006846904728E004212846FFF7F1F818B3FD
:1059E0004FF484712846FFF7E0F8E8B121462846D5
:1059F000FFF768FD616AA069884215D1E06938B196
:105A0000E268616AA0612069E6616662E06008E0C0
:105A100094F8290000B96F60C5F80883A661E268B0
:105A2000616A2046FFF767FD4FF48E7841462846AD
:105A3000FFF7BBF878B1206A6169884202D294F816
:105A4000280020B341462846FFF7B4F8616911B138
:105A50002046FFF733FF4FF4A27841462846FFF770
:105A6000A4F8002818D041462846FFF7A3F894F878
:105A7000290000B12F60A06900280DD0A661E2685E
:105A8000616A04B02046BDE8F047FFF734BD214607
:105A90002846FFF703FFDEE7BDE8FF871FB50A468C
:105AA00001788DF8001041680191017A8DF8081095
:105AB000C0680390044850F82210083850F822209B
:105AC000684690471FBD00004C0000202DE9FF41B3
:105AD0000C464FF4927705463946FFF777F80026D3
:105AE000C0B139462846FFF776F802208DF800004D
:105AF000D5F88004C5F880040390D5F83C058DF8EE
:105B00000800E0680190A661E661D4E900126846E9
:105B1000904723E04FF4887739462846FFF756F838
:105B2000E0B139462846FFF756F8D5F83C15A0698C
:105B3000884213D1E06960B1E268D5F8000220F034
:105B40002000C5F80002E069A0612069E661E0601C
:105B500001E0A661E2682046FFF7D8FC4FF4A27787
:105B600039462846FFF732F860B139462846FFF734
:105B700032F8A06930B1A661D5F83C152046E2683C
:105B8000FFF7C4FC4FF4907739462846FFF71EF81C
:105B9000002813D039462846FFF71DF86069002811
:105BA0000CD0D5F84C058DF800608DF80800A06881
:105BB00001906661D4E9001268469047BDE8FF8114
:105BC0002DE9F05F8346DDE90A4A994690460D4685
:105BD0000846012703E000BFB0FBF8F07F1C4045FA
:105BE000FAD2B94500D94F465FEACA7012D18CB1DA
:105BF0005FEA8A7002D5B9F1000F01D0202607E0D4
:105C0000302605E031465846641EFAF797FF0CB17E
:105C1000A742F7D35FF00106B9F1010F02D9A9F14C
:105C2000010903E0B5FBF6F0404502D306FB08F698
:105C3000F2E7DFF83C9000BFB5FBF6F000FB16552D
:105C400019F800105846FAF779FFB6FBF8F6002E5F
:105C5000F2D15FEACA7009D0002C07D0A74205D262
:105C600020215846641EFAF769FFF5E7BDE8F09F6A
:105C70002C6000000A494A788B78521CD2B29342B9
:105C800000D100220B78934201D1002070470270AE
:105C9000487800EB400001EBC000001D7047000099
:105CA000C00500201CB5002913D08268127C8A42EE
:105CB0000FD008A3D3E90023CDE9002301F12F027F
:105CC0008DF803208268117400696A4603A1FDF70C
:105CD00099FF1CBD1B5B34006D00000025730000A4
:105CE0001CB5826899B1D27B8A420FD00CA2D2E94E
:105CF0000032CDE9003201F12F028DF805208268D3
:105D0000D17300696A4608A1FDF77CFF1CBDD17301
:105D1000006902B0054ABDE8104003A1FDF772BF5B
:105D20001B5B313B33006D0025730000E05F00001A
:105D3000A0010020C00100203F0000000002002060
:105D4000180200200F0000002802002000000000C0
:105D50000020004000000000002000400000000083
:105D60001860000040020020305D0000405D00002F
:105D7000345D00004C5D0000E8610000605D0000E3
:105D80006C0200201800002000000020686A00005B
:105D90000D000000FFFFFFFFFFFFFFFFFFFFFFFF02
:105DA000FFFFFFFF00000000000000000000D60120
:105DB0000701000000000000BC5D000088620000D8
:105DC0005862000000000000ED1E0000806200002C
:105DD0006862000000000000011F000090620000E7
:105DE000F861000000000000B91F00000000000082
:105DF000000000000000000000000000B062000091
:105E000098620000B45D0000951E0000B54C0000D3
:105E10001150000000000000000000000000000021
:105E20000338FDD87047000000000000305E00001D
:105E3000DC620000B8620000000000005930000081
:105E40000000000000000000000000000000000052
:105E5000E4620000EC620000285E0000593000009F
:105E6000FD3F0000E13F0000C53F000000000000D2
:105E7000745E0000CC630000B4630000000000000A
:105E800085330000D06300009C6300000000000028
:105E9000AF33000000000000000000000000000020
:105EA0000000000000000000AC5E0000CC630000B9
:105EB000D46300000000000071340000D0630000D3
:105EC00030640000000000009B340000000000006F
:105ED00000000000000000000000000000000000C2
:105EE000E45E00009C64000070640000000000009C
:105EF00061320000A464000044640000000000005F
:105F000091320000000000000000000000000000CE
:105F100000000000000000001C5F0000F0640000B2
:105F2000D06400006C5E00001D330000E8640000D7
:105F3000AC640000A45E0000D9330000F8640000E7
:105F4000C0640000DC5E0000F531000000000000CD
:105F50000000000000000000000000000000000041
:105F6000645F000044650000006500000000000060
:105F700001360000000000000000000000000000EA
:105F8000000000005C6500004C650000000000009F
:105F90006D3100008865000064650000145F00003A
:105FA000B1310000A06500008C6500000000000019
:105FB000C534000048660000A86500005C5F000072
:105FC0003D3500000000000000000000000000005F
:105FD0001B37001B38001B45002C20001B5B4A00B0
:105FE0001B5B6D00082008001B5B4B00202D200070
:105FF0001B5B48001B5B366E001B5B324A000000D7
:106000000338FDD870471B5B3F336C002D682C2094
:106010002D2D68656C70000055170000AB1700004F
:10602000E9160000C1170000A1170000303132331B
:106030003435363738394142434445460000000084
:1060400044600000DC6200005466000000000000B4
:106050007148000000000000000000000000000087
:106060000000000078660000EC6200003C60000068
:106070007148000001000000ED2E0000010000004A
:1060800099550000000000008C6000001C680000B2
:10609000A8670000746000002D280000146800004C
:1060A000246700007C6000002D2800004468000088
:1060B0002468000000000000052A00005868000065
:1060C00034680000000000000D2A0000DC620000BF
:1060D0004868000000000000B12A00000000000035
:1060E00000000000000000000000000060680000E8
:1060F0006468000084600000D52700000040404034
:10610000404040404040414141414140404040408A
:106110004040404040404040404040404005020236
:1061200002020202020202020202020202202020F5
:106130002020202020202002020202020202909051
:10614000909090901010101010101010101010104F
:1061500010101010101010100202020202028888A3
:1061600088888888080808080808080808080808AF
:106170000808080808080808020202024000000097
:10618000FD600000457865637574653A203C666C77
:10619000617368202D683E20666F72206D6F726596
:1061A00020696E666F726D6174696F6E206F722008
:1061B0007072657373207468652054616220627523
:1061C00074746F6E20746F2073656520616C6C2031
:1061D000617661696C61626C6520636F6D6D616E83
:1061E00064732E0D0A000000756172745F636C6940
:1061F0003A7E2420000000005772697465206461B3
:10620000746120746F20666C6173682E0A4C696D2E
:1062100069746174696F6E733A0A2D206D617869D3
:106220006D756D20313620656E74726965732C0A48
:106230002D206561636820656E7472792069732012
:106240006D6178696D756D20363220636861727397
:10625000206C6F6E672E0000457261736520666C5E
:106260006173682E000000005265616420646174EF
:10627000612066726F6D20666C6173682E0000008D
:106280007265616400000000657261736500000062
:106290007772697465000000466C61736820616301
:1062A0006365737320636F6D6D616E642E00000013
:1062B000666C6173680000005072696E74207374BC
:1062C00061747573206F662062616C6C6F63206906
:1062D0006E7374616E6365732E0000007374617475
:1062E0007573000062616C6C6F630000436F6D6DCD
:1062F000616E647320666F722042414C4C4F4320A4
:106300006D616E6167656D656E74000025730D0AC1
:10631000092D20456C656D656E742073697A653A48
:10632000092564202B202564206279746573206F11
:106330006620646562756720696E666F726D617450
:10634000696F6E0D0A092D2055736167653A09253D
:1063500075252520282575206F7574206F662025EA
:106360007520656C656D656E7473290D0A092D20A5
:106370004D6178696D756D3A0925752525202825AB
:1063800075206F7574206F6620257520656C656DAE
:10639000656E7473290D0A0D0A000000456E616276
:1063A0006C6520636F6C6F7265642073796E7461C5
:1063B000782E000044697361626C6520636F6C6FB6
:1063C0007265642073796E7461782E006F66660062
:1063D0006F6E000044697361626C6520434C492014
:1063E0006563686F2E204172726F777320616E64EF
:1063F00020627574746F6E733A204261636B7370C0
:106400006163652C2044656C6574652C20456E6461
:106410002C20486F6D652C20496E73657274206165
:106420007265206E6F742068616E646C65642E0006
:10643000456E61626C6520434C49206563686F2E30
:106440000000000047657420434C49207374617458
:1064500069737469637320666F7220746865204C79
:106460006F67676572206D6F64756C652E00000044
:10647000526573657420434C492073746174697369
:106480007469637320666F7220746865204C6F674F
:10649000676572206D6F64756C652E00726573653B
:1064A0007400000073686F7700000000546F676726
:1064B0006C6520434C49206563686F2E0000000026
:1064C000434C4920737461746973746963732E005B
:1064D000546F67676C6520636F6C6F7265642073BF
:1064E000796E7461782E00006563686F00000000AB
:1064F000636F6C6F727300007374617473000000DB
:10650000417373756D652038302063686172732044
:1065100073637265656E20776964746820616E6468
:106520002073656E64207468697320736574746980
:106530006E6720746F20746865207465726D696E73
:10654000616C2E0064656661756C7400436C6561F6
:10655000722073637265656E2E000000636C656166
:106560007200000055736566756C2C206E6F742088
:10657000556E69782D6C696B6520434C4920636FBB
:106580006D6D616E64732E00636C6900436F6D6D99
:10659000616E6420686973746F72792E0000000068
:1065A000686973746F727900436F6E736F6C6520E6
:1065B00067657473207465726D696E616C207363B6
:1065C0007265656E2073697A65206F7220617373DE
:1065D000756D657320383020696E206361736520A6
:1065E00074686520726561646F7574206661696C9A
:1065F000732E204974206D75737420626520657850
:106600006563757465642061667465722065616395
:1066100068207465726D696E616C20776964746856
:10662000206368616E676520746F20656E73757294
:106630006520636F7272656374207465787420647A
:106640006973706C61792E00726573697A650000F8
:10665000202000005072696E742073746174757329
:10666000206F6620717565756520696E7374616E43
:106670006365732E0000000071756575650000008C
:1066800025730D0A092D20456C656D656E742073A8
:10669000697A653A0925640D0A092D2055736167E9
:1066A000653A092575252520282575206F757420E4
:1066B0006F6620257520656C656D656E7473290D98
:1066C0000A092D204D6178696D756D3A092575258A
:1066D0002520282575206F7574206F66202575206C
:1066E000656C656D656E7473290D0A092D204D6FFB
:1066F00064653A090925730D0A0D0A006E6F6E650F
:10670000000000007761726E696E670064656275F3
:1067100067000000696E666F000000006572726FAE
:1067200072000000276C6F6720656E61626C6520E7
:106730003C6C6576656C3E203C6D6F64756C655F86
:10674000303E202E2E2E20203C6D6F64756C655FD0
:106750006E3E2720656E61626C6573206C6F677397
:1067600020757020746F20676976656E206C657681
:10677000656C20696E207370656369666965642065
:106780006D6F64756C65732028616C6C2069662080
:106790006E6F206D6F64756C6573207370656369CF
:1067A00066696564292E0000276C6F672064697331
:1067B00061626C65203C6D6F64756C655F303E2076
:1067C0002E2E203C6D6F64756C655F6E3E272064D5
:1067D000697361626C6573206C6F677320696E20EA
:1067E000737065636966696564206D6F64756C6557
:1067F000732028616C6C206966206E6F206D6F6459
:10680000756C657320737065636966696564292EAC
:1068100000000000656E61626C6500006469736170
:10682000626C6500526573756D65206C6F67676992
:106830006E67000048616C74206C6F6767696E67F3
:1068400000000000676F00004C6F6767657220737F
:10685000746174757300000068616C74000000005E
:106860006C6F6700436F6D6D616E647320666F724D
:1068700020636F6E74726F6C6C696E67206C6F67EB
:10688000676572001B5B313B33306D001B5B306D05
:10689000000000001B5B313B33316D001B5B313B63
:1068A00033326D001B5B313B33336D001B5B313B7F
:1068B00033346D001B5B313B33356D001B5B313B6B
:1068C00033366D001B5B313B33376D007175657579
:1068D000652E6D5F636C695F756172745F6C6F6765
:1068E0005F6261636B656E645F71756575650000FD
:1068F00062616C6C6F632E6D5F636C695F75617252
:10690000745F636D645F686973745F6D656D6F62FA
:106910006A0000006D5F636C695F756172745F6C23
:106920006F675F6261636B656E645F7175657565E6
:10693000000000006D5F636C695F756172745F6376
:106940006D645F686973745F6D656D6F626A000086
:10695000636C6F636B000000434C4F434B000000BF
:1069600050525300554152540000000055415254BA
:1069700045000000636C695F75617274000000007F
:106980007077725F6D676D740000000062616C6CFF
:106990006F632E6C6F675F6D656D706F6F6C00005D
:1069A000617070006C6F675F6D656D706F6F6C000C
:1069B000BC6A000000000020A0010000A404000048
:1069C000106B0000A0010020102A0000D407000076
:1069D00000000000FC5D000000000000505E0000B0
:1069E00000000000845F000000000000945F0000D1
:1069F00000000000A45F000000000000B45F000081
:106A0000000000006460000000000000EC60000076
:106A1000CC68000000000003F068000000000003E4
:106A200050690000000000005869000000000000EC
:106A300060690000000000006469000000000000C0
:106A40006C69000000000000746900000000000094
:106A500080690000000000008C6900000000000355
:106A6000A06900000000030338000020300000206F
:106A700038000020CC0300202801002034690000E9
:106A800030000000B0000020A8000020B00000206E
:106A9000CC06002088010020A46900001800000036
:106AA000C0030020AC03002004000000040000002C
:106AB00001000000146900001C010020138003B3D2
:106AC000201723785D23053AA3605E0356A06A234E
:106AD00050661AFC04231C671A04041A14045A0C86
:106AE00004291429102920291C011CE940238C6841
:106AF0001A84041A94041A9C041AA4041AAC041AE2
:106B0000B4041ABC041AC4041104A490D0030000F5
:0400000500000201F4
:00000001FF
